:100000000EC027C025C024C023C022C021C020C0EC
:100010001FC01EC01DC01CC01DC01AC019C01124A5
:100020001FBECFEDCDBF10E0A0E6B0E0E0E5F6E00A
:1000300002C005900D92A036B107D9F710E0A0E6F6
:10004000B0E001C01D92A036B107E1F702D1FEC2B7
:10005000D7CF18951895C29A000086B3C29880959C
:1000600084700895C29A00008BB780648BBF85B7F7
:10007000877E806185BF85B7806285BF889585B79B
:100080008F7D85BF8BB78F7B8BBFC298089540E073
:1000900061E083E007D0C29A000086B3C29882FF75
:1000A000F6CF08953FB7F894A895982F9770292F09
:1000B000206483FF02C0292F206681B5886181BD3D
:1000C00021BD3FBF85B7877E806185BF90E022C09C
:1000D00085B7806285BF889585B78F7D85BF4423AE
:1000E000C1F0C29A000086B3C29882FD12C087B3E5
:1000F000877E87BBCCDF28E088E190E00FB6F894DC
:10010000A89581BD0FBE21BD85B7877E806185BF63
:10011000FFCF9F5F9617E0F281B5886181BD11BC6A
:100120000895CF92DF92EF92FF920F931F93CF9398
:10013000DF938C016B01FC01108284E0E82EFF2428
:10014000C0E0D0E040E061E082E0ACDFC29A0000B5
:1001500096B3C29890959470EE2069F0992369F453
:10016000F80180818F5F8083F601D183C083FF24F3
:10017000C0E0D0E008C0992331F0FFEFCF3FDF07A8
:1001800019F0219601C0F394E92E8CE08F15D0F67A
:10019000DF91CF911F910F91FF90EF90DF90CF9063
:1001A0000895FF920F931F93F82E062F142F2223EA
:1001B00091F041E068E083E075DF87B3886187BB39
:1001C00041E064E083E06EDF87B3877E87BB41E078
:1001D0006AE083E067DFE199FECF82E090E0982F4C
:1001E0008EBBE09A8DB3813021F487B3886187BBE1
:1001F0000DC0E199FECF9EBBE09A8DB3823029F409
:10020000BB9A41E061E083E04DDFBC9A41E062E0EF
:1002100083E048DF20E04AEF50E004C0CA010197C4
:10022000F1F72F5F2117D0F341E0602F8F2D3ADFD8
:1002300087B3877E87BBE199FECF80E090E08EBBDD
:10024000E09A6DB341E083E02DDF1F910F91FF90A5
:1002500008950F931F93DF93CF9300D00F92CDB7E4
:10026000DEB7A89584B7877F84BF88E10FB6F8947E
:1002700081BD11BC0FBE479A8FE080BD7894F2DE3D
:10028000BE016E5F7F4FCE0101964BDFE199FECF3D
:1002900081E090E0982F8EBBE09A2DB38981813068
:1002A00009F054C08A819B81099750F187B3886116
:1002B00087BB00E010E006C041E061E082E0F2DED2
:1002C0000F5F1F4F8A819B819695879508171907A5
:1002D00098F387B3877E87BB00E010E006C041E05B
:1002E00061E082E0DFDE0F5F1F4F8A819B819C010E
:1002F00036952795821B930B08171907B8F6EFCF91
:10030000222329F440E062E080E04BDF02C021308C
:1003100029F420E045E063E080E043DF20E040E0B6
:1003200069E080E03EDF20E040E062E280E039DF2B
:1003300020E040E060E183E034DF20E040E060E482
:1003400083E02FDF20E040E060EF22C0823009F040
:100350004DC08A819B810997F0F4222329F44AE059
:1003600061E080E01EDF02C0213051F420E048E06F
:1003700062E080E016DF20E040E065E080E011DF31
:1003800020E040E061E180E00CDF20E040E068E058
:1003900083E007DF3FC1222351F44AE061E080E0BF
:1003A00000DF20E040E062E080E0FBDE02C02130C0
:1003B00079F420E048E062E080E0F3DE20E045E010
:1003C00063E080E0EEDE20E040E065E080E0E9DE32
:1003D00020E040E069E080E0E4DE20E040E061E130
:1003E00080E0DFDE20E040E062E2CDCF833009F044
:1003F00045C08A819B810997A0F420E040E068E035
:1004000083E0CFDE20E040E060E283E0CADE20E06F
:1004100040E068E783E0C5DE20E040E060EF84E094
:1004200027C020E040E068E083E0BBDE20E040E061
:1004300060E183E0B6DE20E040E060E283E0B1DE30
:1004400020E040E060E483E0ACDE20E040E068E7EC
:1004500083E0A7DE20E040E060EF83E0A2DE20E062
:1004600040E060EF84E09DDE20E040E060EF85E06A
:1004700098DE20E040E060EF86E08BCF843009F02A
:1004800057C08A819B810997D0F4223028F421E05B
:100490004AE061E080E085DE21E040E062E083E068
:1004A00080DE21E040E068E083E07BDE21E040E0A8
:1004B00060E283E076DE21E040E068E732C022308F
:1004C00028F421E04AE061E080E06BDE21E04AE0D0
:1004D00066E080E066DE21E040E062E083E061DE2D
:1004E00021E040E064E083E05CDE21E040E068E0A1
:1004F00083E057DE21E040E060E183E052DE21E06E
:1005000040E060E283E04DDE21E040E060E483E033
:1005100048DE21E040E068E783E043DE21E040E0A0
:1005200060EF83E03EDE21E040E060EF84E031CF29
:10053000863031F4E199FECF1CBA80E090E062C0D1
:10054000873041F4E199FECF1CBA80E090E08EBB89
:1005500084E05AC0883041F4E199FECF1CBA80E0B3
:1005600090E08EBB86E050C0893041F4E199FECF27
:100570001CBA80E090E08EBB8AE046C08A3041F42D
:10058000E199FECF1CBA80E090E08EBB80E13CC0D8
:100590008B3041F4E199FECF1CBA80E090E08EBB35
:1005A00088E132C08C3029F4E199FECF1CBA9EBBA1
:1005B00016C08D3029F4E199FECF1CBA9EBB19C03C
:1005C0008E3029F4E199FECF1CBA9EBB1CC08F303F
:1005D00041F4E199FECF1CBA82E090E08EBB1DBAD7
:1005E00014C0803141F4E199FECF1CBA82E090E062
:1005F0008EBB81E009C0813169F4E199FECF1CBA5C
:1006000082E090E08EBB82E08DBB0FB6F894E29A58
:10061000E19A0FBE88E028E130E00FB6F894A89583
:1006200021BD0FBE81BD85B7877E806185BFFFCFAD
:1006300088E028E130E00FB6F894A89521BD0FBE00
:1006400081BD85B7877E806185BFFFCFF894FFCFDE
:00000001FF
